:1000000010C02AC029C028C027C026C025C024C0CF
:1000100023C022C021C020C01FC01EC01DC01CC0E4
:100020001BC011241FBECFE5D2E0DEBFCDBF10E064
:10003000A0E6B0E0E0E7F2E002C005900D92A23643
:10004000B107D9F710E0A2E6B0E001C01D92A336D7
:10005000B107E1F763D00AC1D3CF80E88ABB8FE153
:1000600087BB089590916000981789F098B3987FA6
:1000700098BBDF9828B3982F9770922B98BB2BB31F
:10008000982F92959078922B9BBB80936000089557
:100090001F93CF93DF93EC011091600080E0E2DFCB
:1000A00020E030E003C000002F5F3F4F2C173D07DA
:1000B000D4F3812FD7DFDF91CF911F91089585E091
:1000C000D1DF8FE39DE0A3E081509040A040E1F7B5
:1000D00000C0000080E0C6DFA7EAB1E61197F1F7A3
:1000E00000C000008AE0BEDF8FE39DE0A3E0815006
:1000F0009040A040E1F700C0000080E0B3DF089529
:1001000029B330E02370307080916200882321F0A1
:1001100083E090E028273927C9010895CF93DF9322
:1001200083E294EF0197F1F700C0000096DFA1EEA3
:10013000B4E01197F1F700C0000080E093DFCD99A3
:1001400013C02FE936E841E0215030404040E1F74C
:1001500000C00000B4DF8FE996E8A1E08150904034
:10016000A040E1F700C00000CE9903C081E0809379
:100170006200A3ECB9E01197F1F700C00000D69A35
:10018000E3ECF9E03197F1F700C000008BB390E4A5
:1001900089278BBB2FE936E841E0215030404040B1
:1001A000E1F700C000008BB389278BBB8FE996E88D
:1001B000A1E081509040A040E1F700C0000090E431
:1001C00009C08BB389278BBBA3EDB0E31197F1F77F
:1001D00000C00000CD99F5CF2FE33DE043E0215072
:1001E00030404040E1F700C00000C0E0D0E0219680
:1001F000C630D1052CF08AE090E04ADFC0E0D0E0C4
:100200007FDF823018F0823069F514C080E02ADF89
:10021000DE9A8AE027DF8FE295E70197F1F700C0C9
:10022000000080E01FDF86E01DDFA7EAB1E611973E
:10023000F1F713C080E016DFDE9A8AE013DFEFE209
:10024000F5E73197F1F700C0000080E00BDF89E0AF
:1002500009DF87EA91E60197F1F700C0000080E02E
:1002600001DFC5CF85E0FEDED698C1CFF894FFCF81
:02027000FF008D
:00000001FF
